:020000040000FA
:0600000000008A01BF2888
:080008007108FC3E03190B28EE
:10001000FF3E031D1E28F71C1E2806083039303A03
:10002000F60003191E287516761A7514F61AF514BB
:1000300077181E280630F100FD21F30128308100D9
:100040000B1124202C2009008A017208820737280E
:1000500038283C28422852288A0171088207DB2868
:10006000E628EF28FA280A291C2929293929080015
:1000700058208618F20A0800861808003030F4006C
:10008000F20A0800F40B4828F20AF001F7210800F0
:10009000861C0800F70A7708FC3E0319F701582070
:1000A000F2030800861C0800F201F1016820080034
:1000B0005B20F000F729770882070134023404340A
:1000C0000834030183169B001C141A0883120800CD
:1000D000770883169B0183169A001C1555309D00E6
:1000E000AA309D009C1483128C1F74288C13080066
:1000F00001306220813A031D832802306220693A70
:10010000031D8328003483160130F700682083160E
:1001100001309B0081306B2083169B0A69306B2075
:100120008312FF34F8009D20F80B93280800F90093
:1001300064309220F90B98280800C6300000FF3E7A
:10014000031D9E280000000000000800F701003099
:100150008A00B320F000F721F70A02309720F00858
:10016000031DA92808007708820704340A341134D3
:100170000A3404340E341F341B3411340034073075
:100180009F008316E0308500FE3086000730810036
:100190008312A62001309000F101F201F301F40175
:1001A000F001FB2178206120F700283081000B113D
:1001B0008B168B17DA28F208031D0800FB2186181E
:1001C0000800F10AF3013030F40008008618ED2829
:1001D000F40B0800F101F20A0800F10A0800060811
:1001E0003039303A0319F8280A30F000F7210800B6
:1001F000F10A080006083039303A03190129F103E1
:100200000800F10AF001F501F708031D08000330AA
:1002100086000800730803190F29F3030800F01A79
:1002200017291230F3000314F00DF7210800F10A2A
:100230000E083F39F3000800730803192129F3035E
:100240000800F001F721F71CFB21F10A1830F30038
:100250000800730803192E29F30308007508031911
:100260003729F000F721FF30F300F10A0800F1010F
:100270000800730803194029F303861CF1010800E4
:10028000F001F721F101080053346C346F347434F9
:100290002034433461347234203452346134633452
:1002A00065342034533474346134723474342034FB
:1002B00043346F346E34743472346F346C346C3451
:1002C000653472345034433442342034523465340B
:1002D0007634203432342E3420345734653462344A
:1002E0002034723465346C3465346134733465346D
:1002F000203466346F3472342034533463346134C0
:100300006C34653478347434723469346334203432
:10031000533470346F347234743420346F346E3428
:100320006C34793443346F347034793472346934D2
:100330006734683474342034283443342934203406
:1003400032343034303436342D3432343034313485
:1003500031342E342034503465347434653472347E
:100360002034473472346934663466346934743402
:1003700068347334723473346334403470346934A1
:100380006334703472346F346A3465346334743473
:1003900073342E346F3472346734463472346534B7
:1003A0006534203466346F347234203470346534EC
:1003B000723473346F346E3461346C342C342034C2
:1003C0006E346F346E342D3463346F346D346D3469
:1003D000653472346334693461346C342034753478
:1003E0007334653420346F346E346C34793470086F
:0E03F000FF3A850008000610080006140800F9
:02400E00103F61
:00000001FF
